:100000002500660067003F0C0600370C0700000C57
:100010000200000BE2019A08E90800085A08350BB3
:10002000430B510B290B5E0BFF0FFF0FFF0FFF0F51
:10003000FF0FFF0FFF0FFF0FFF0FFF0FFF0FFF0F50
:10004000FF0FFF0FFF0FFF0FFF0FFF0FFF0FFF0F40
:10005000FF0FFF0FFF0FFF0FFF0FFF0FFF0FFF0F30
:10006000FF0FFF0FFF0FFF0FFF0FFF0FFF0FFF0F20
:10007000FF0FFF0FFF0FFF0FFF0FFF0FFF0FFF0F10
:10008000FF0FFF0FFF0FFF0FFF0FFF0FFF0FFF0F00
:10009000FF0FFF0FFF0FFF0FFF0FFF0FFF0FFF0FF0
:1000A000FF0FFF0FFF0FFF0FFF0FFF0FFF0FFF0FE0
:1000B000FF0FFF0FFF0FFF0FFF0FFF0FFF0FFF0FD0
:1000C000FF0FFF0FFF0FFF0FFF0FFF0FFF0FFF0FC0
:1000D000FF0FFF0FFF0FFF0FFF0FFF0FFF0FFF0FB0
:1000E000FF0FFF0FFF0FFF0FFF0FFF0FFF0FFF0FA0
:1000F000FF0FFF0FFF0FFF0FFF0FFF0FFF0FFF0F90
:10010000FF0FFF0FFF0FFF0FFF0FFF0FFF0FFF0F7F
:10011000FF0FFF0FFF0FFF0FFF0FFF0FFF0FFF0F6F
:10012000FF0FFF0FFF0FFF0FFF0FFF0FFF0FFF0F5F
:10013000FF0FFF0FFF0FFF0FFF0FFF0FFF0FFF0F4F
:10014000FF0FFF0FFF0FFF0FFF0FFF0FFF0FFF0F3F
:10015000FF0FFF0FFF0FFF0FFF0FFF0FFF0FFF0F2F
:10016000FF0FFF0FFF0FFF0FFF0FFF0FFF0FFF0F1F
:10017000FF0FFF0FFF0FFF0FFF0FFF0FFF0FFF0F0F
:10018000FF0FFF0FFF0FFF0FFF0FFF0FFF0FFF0FFF
:10019000FF0FFF0FFF0FFF0FFF0FFF0FFF0FFF0FEF
:1001A000FF0FFF0FFF0FFF0FFF0FFF0FFF0FFF0FDF
:1001B000FF0FFF0FFF0FFF0FFF0FFF0FFF0FFF0FCF
:1001C000FF0FFF0FFF0FFF0FFF0FFF0FFF0FFF0FBF
:1001D000FF0FFF0FFF0FFF0FFF0FFF0FFF0FFF0FAF
:1001E000FF0FFF0FFF0FFF0FFF0FFF0FFF0FFF0F9F
:1001F000FF0FFF0FFF0FFF0FFF0FFF0FFF0FFF0F8F
:1002000011091B0C29001009E902030B4707130A07
:100210001B0C29001009E9020A0B3F0C46012F00B4
:10022000370C47013000100C29001009E902150BAA
:100230000F090D0C2400040C28006C000002EC01D6
:1002400000021209A402E8021E0B0C021209080B9C
:10025000FF0F2B00080C29006B030306310B0F095D
:10026000320B1009E9022C0B1009080C2700CA0CEC
:100270002A00EA02390B000C2700CA0C2A00EA0205
:100280003F0B0008FF0F000C2700CA0C2A00EA02EF
:10029000470B080C2700CA0C2A00EA024D0B000885
:1002A000FF0F0D0C2400680008020A092000A402B8
:1002B000A802040C88004307540B00080F090F091B
:0602C00047071009130AB4
:021FFE00D40FFE
:00000001FF
